:100000000C9462000C948A000C948A000C948A0070
:100010000C948A000C948A000C948A000C948A0038
:100020000C948A000C948A000C948A000C948A0028
:100030000C948A000C948A000C948A000C948A0018
:100040000C94B2010C948A000C948A000C948A00DF
:100050000C948A000C948A000C948A000C948A00F8
:100060000C948A000C948A000000000024002700F1
:100070002A0000000000250028002B0000000000DE
:1000800023002600290004040404040404040202DA
:100090000202020203030303030301020408102007
:1000A0004080010204081020010204081020000012
:1000B0000008000201000003040700000000000027
:1000C0000000540411241FBECFEFD8E0DEBFCDBF27
:1000D00011E0A0E0B1E0E4E4FDE002C005900D9283
:1000E000AE32B107D9F721E0AEE2B1E001C01D9216
:1000F000A736B207E1F710E0C2E6D0E004C02197CE
:10010000FE010E949A06C136D107C9F70E94FC0180
:100110000C94A0060C940000833081F028F4813008
:1001200099F08230A9F008958730A9F08830C9F09D
:100130008430B1F4809180008F7D03C08091800075
:100140008F7780938000089584B58F7784BD08955C
:1001500084B58F7DFBCF8091B0008F778093B00006
:1001600008958091B0008F7DF9CFCF93DF93282F32
:1001700030E0F901E255FF4F8491F901E656FF4F57
:10018000D491F901EA57FF4FC491CC23A1F081111A
:100190000E948C00EC2FF0E0EE0FFF1FE458FF4FA1
:1001A000A591B491EC91ED2381E090E009F480E019
:1001B000DF91CF91089580E090E0FACF1F93CF9325
:1001C000DF93282F30E0F901E255FF4F8491F901C8
:1001D000E656FF4FD491F901EA57FF4FC491CC2363
:1001E000A9F0162F81110E948C00EC2FF0E0EE0F89
:1001F000FF1FEE58FF4FA591B4918FB7F894EC9183
:10020000111108C0D095DE23DC938FBFDF91CF9111
:100210001F910895DE2BF8CFCF93DF9390E0FC0180
:10022000E656FF4F24918A579F4FFC018491882303
:10023000C9F090E0880F991FFC01E859FF4FA59184
:10024000B491FC01EE58FF4FC591D49161110DC0DE
:100250009FB7F8948C91209582238C9388812823D2
:1002600028839FBFDF91CF910895623051F49FB7EB
:10027000F8943C91822F809583238C93E8812E2BD8
:10028000EFCF8FB7F894EC912E2B2C938FBFEACF42
:100290008E50806480937C0080917A00806480938B
:1002A0007A0080917A0086FDFCCF80917800909151
:1002B00079000895873691058CF0853321E0920707
:1002C0007CF0833022E092076CF0813D22E09207BF
:1002D0005CF08F39934054F085E0089580E00895F4
:1002E00081E0089582E0089583E0089584E0089510
:1002F000CF92DF92EF92FF92CF93C1E0C0934C0177
:1003000080910801909109019093460180934501E5
:10031000109247018FB7F894C0906301D0906401A8
:10032000E0906501F09066018FBF61E08BE00E9474
:10033000DE0061E083E00E94DE00C093470185E0BB
:10034000C80ED11CE11CF11CC0924801D092490199
:10035000E0924A01F0924B01CF91FF90EF90DF9035
:10036000CF9008951F920F920FB60F9211242F93E2
:100370003F938F939F93AF93BF938091630190912D
:100380006401A0916501B09166013091620123E0A2
:10039000230F2D3758F50196A11DB11D2093620141
:1003A0008093630190936401A0936501B09366010B
:1003B00080915E0190915F01A0916001B091610117
:1003C0000196A11DB11D80935E0190935F01A093E2
:1003D0006001B0936101BF91AF919F918F913F9167
:1003E0002F910F900FBE0F901F90189526E8230FA6
:1003F0000296A11DB11DD2CF789484B5826084BDD0
:1004000084B5816084BD85B5826085BD85B5816018
:1004100085BD80916E00816080936E001092810096
:100420008091810082608093810080918100816051
:100430008093810080918000816080938000809112
:10044000B10084608093B1008091B000816080939E
:10045000B00080917A00846080937A0080917A0065
:10046000826080937A0080917A00816080937A0024
:1004700080917A00806880937A001092C10060E0D9
:1004800089E00E940C0161E08BE00E940C0161E0B8
:1004900083E00E940C0162E084E00E940C0160E0B5
:1004A00081E10E940C0160E08BE00E94DE0060E0D0
:1004B00083E00E94DE0093E0892E912CA12CB12CC8
:1004C00000E010E0772473948FB7F894C090630134
:1004D000D0906401E0906501F09066018FBF8EE0DE
:1004E0000E944801EC0183E10E9448019C01CE0179
:1004F000DD0FAA0BBB0B032E000C440B550B820F18
:10050000931FA41FB51FB7FD78C1811524E0920782
:10051000A105B1050CF074C10E945A01E82FF0E06A
:10052000EE0FFF1FE65FFE4F8081918190930901DE
:10053000809308018FE00E9448010E945A0194E0D4
:10054000899FF0011124EA5EFE4F80819181A28192
:10055000B3818093040190930501A0930601B093A9
:10056000070180E10E944801C2970CF04CC17092D3
:100570005D0181E10E94B500EC01019709F068C0BE
:1005800080913F0190914001892B09F061C02FB704
:10059000F8948091630190916401A0916501B091FC
:1005A00066012FBF40913B0150913C0160913D019C
:1005B00070913E011C012D01241A350A460A570A82
:1005C000B201A10180933B0190933C01A0933D01B6
:1005D000B0933E0180913A0124E0829FF001112402
:1005E000E25DFE4F40835183628373838F5F83306C
:1005F00008F02FC180933A0160913201709133016C
:10060000809134019091350120912E0130912F017C
:100610004091300150913101620F731F841F951F6B
:1006200020913601309137014091380150913901C4
:10063000620F731F841F951FA50194010E94680417
:100640002093410130934201409343015093440170
:10065000D0934001C0933F0189E00E94B500EC01B6
:1006600090935C0180935B01019761F48091590143
:1006700090915A01892B31F480914C01811102C073
:100680000E947801D0935A01C093590184E00E94DE
:10069000B500109257011092580190915601891798
:1006A00051F080935601C0925101D0925201E092D4
:1006B0005301F09254018091510190915201A09107
:1006C0005301B0915401B701A601481B590B6A0BA5
:1006D0007B0B80914D0190914E01A0914F01B09103
:1006E000500184179507A607B707B0F490915501FC
:1006F00080915601981781F080935501911103C0A4
:1007000021E0813009F020E020935701913009F475
:10071000811190E09093580180915801882331F025
:1007200080914C01811102C00E94780180914C019E
:10073000882309F4A2C08091480190914901A091B9
:100740004A01B0914B01C816D906EA06FB0608F427
:1007500094C080914701882309F496C060E08BE043
:100760000E94DE0060E083E00E94DE0010924701FC
:1007700080914501909146010197909346018093A5
:100780004501181619060CF076C080915D0188238A
:1007900009F462C06091410170914201809143016E
:1007A00090914401611571058105910509F454C0CA
:1007B0000E949F052091040130910501409106019E
:1007C000509107010E942D060E946905DC01CB01B2
:1007D0000597A109B109B7FF03C080E090E0DC01F3
:1007E000C80ED91EEA1EFB1EC0924801D0924901D4
:1007F000E0924A01F0924B0140C090E080E08CCE44
:100800008FEF93E089CE10925D0180E10E94480154
:10081000BC01990F880B990B0E94A10520E030E0E4
:1008200048E453E40E942D0620E030EC4FE754E406
:100830000E94F70420E030E040EA52E40E948B047A
:100840006093000170930101809302019093030172
:1008500090CE10923A01D0CE20910001309101014A
:10086000409102015091030160E070E68AE697E44E
:100870000E94F7049FCF10924C010115110509F455
:1008800023CE0E94000020CE61E08BE00E94DE00BB
:1008900061E083E00E94DE007092470185E0C80EAF
:1008A000D11CE11CF11CA0CFEDE4F1E084E190E06B
:1008B000A0E0B0E080839183A283B3831482158289
:1008C0001682178281E080878187128613860895B9
:1008D000A1E21A2EAA1BBB1BFD010DC0AA1FBB1F44
:1008E000EE1FFF1FA217B307E407F50720F0A21BB6
:1008F000B30BE40BF50B661F771F881F991F1A9423
:1009000069F760957095809590959B01AC01BD014C
:10091000CF0108955058BB27AA270E94A2040C9427
:10092000F3050E94E50538F00E94EC0520F039F44B
:100930009F3F19F426F40C94E2050EF4E095E7FBD2
:100940000C94DC05E92F0E94040658F3BA176207DD
:1009500073078407950720F079F4A6F50C94260612
:100960000EF4E0950B2EBA2FA02D0B01B9019001CA
:100970000C01CA01A0011124FF27591B99F0593F0E
:1009800050F4503E68F11A16F040A22F232F342F56
:100990004427585FF3CF469537952795A795F040A4
:1009A0005395C9F77EF41F16BA0B620B730B840BB9
:1009B000BAF09150A1F0FF0FBB1F661F771F881F71
:1009C000C2F70EC0BA0F621F731F841F48F48795C9
:1009D00077956795B795F7959E3F08F0B0CF9395BB
:1009E000880F08F09927EE0F9795879508950E9434
:1009F0000B050C94F3050E94EC0558F00E94E505E8
:100A000040F029F45F3F29F00C94DC0551110C945F
:100A100027060C94E2050E94040668F39923B1F3BB
:100A2000552391F3951B550BBB27AA276217730714
:100A3000840738F09F5F5F4F220F331F441FAA1FA8
:100A4000A9F335D00E2E3AF0E0E832D09150504064
:100A5000E695001CCAF72BD0FE2F29D0660F771F12
:100A6000881FBB1F261737074807AB07B0E809F0F8
:100A7000BB0B802DBF01FF2793585F4F3AF09E3F7D
:100A8000510578F00C94DC050C9427065F3FE4F3E5
:100A9000983ED4F3869577956795B795F7959F5FC0
:100AA000C9F7880F911D9695879597F90895E1E00C
:100AB000660F771F881FBB1F621773078407BA076B
:100AC00020F0621B730B840BBA0BEE1F88F7E095C6
:100AD00008950E9470056894B1110C94270608953A
:100AE0000E940C0688F09F5798F0B92F9927B751AC
:100AF000B0F0E1F0660F771F881F991F1AF0BA95C2
:100B0000C9F714C0B13091F00E942606B1E00895F3
:100B10000C942606672F782F8827B85F39F0B93FE5
:100B2000CCF3869577956795B395D9F73EF4909574
:100B30008095709561957F4F8F4F9F4F0895E894F2
:100B400009C097FB3EF490958095709561957F4F15
:100B50008F4F9F4F9923A9F0F92F96E9BB279395C3
:100B6000F695879577956795B795F111F8CFFAF4D3
:100B7000BB0F11F460FF1BC06F5F7F4F8F4F9F4F04
:100B800016C0882311F096E911C0772321F09EE862
:100B9000872F762F05C0662371F096E8862F70E0C8
:100BA00060E02AF09A95660F771F881FDAF7880FA2
:100BB0009695879597F9089597F99F6780E870E073
:100BC00060E008959FEF80EC089500240A941616C3
:100BD000170618060906089500240A94121613062B
:100BE000140605060895092E0394000C11F48823B9
:100BF00052F0BB0F40F4BF2B11F460FF04C06F5FD5
:100C00007F4F8F4F9F4F089557FD9058440F551FAA
:100C100059F05F3F71F04795880F97FB991F61F07E
:100C20009F3F79F087950895121613061406551FF5
:100C3000F2CF4695F1DF08C0161617061806991F61
:100C4000F1CF86957105610508940895E894BB2756
:100C500066277727CB0197F908950E9440060C94E8
:100C6000F3050E94E50538F00E94EC0520F095237D
:100C700011F00C94DC050C94E20511240C94270669
:100C80000E94040670F3959FC1F3950F50E0551F25
:100C9000629FF001729FBB27F00DB11D639FAA27D1
:100CA000F00DB11DAA1F649F6627B00DA11D661F20
:100CB000829F2227B00DA11D621F739FB00DA11D41
:100CC000621F839FA00D611D221F749F3327A00DFB
:100CD000611D231F849F600D211D822F762F6A2F97
:100CE00011249F5750409AF0F1F088234AF0EE0FFC
:100CF000FF1FBB1F661F771F881F91505040A9F729
:100D00009E3F510580F00C94DC050C9427065F3F54
:100D1000E4F3983ED4F3869577956795B795F79564
:100D2000E7959F5FC1F7FE2B880F911D96958795DC
:100D300097F90895EE0FFF1F0590F491E02D0994A7
:040D4000F894FFCF55
:100D44000000A0420000003F010001000300040075
:100D54000600080010000000003F4CA6AA3E000058
:0E0D6400803E68B32A3E0000003E0000803D45
:00000001FF
